:020000040800F2
:1000000000060020E1010008E3010008E301000808
:10001000E3010008E3010008E3010008E301000830
:10002000E3010008E3010008E30100083536000899
:10003000E3010008E3010008E3010008E301000810
:10004000E3010008E3010008E3010008E301000800
:10005000E3010008E3010008E1380008093900085D
:10006000313900085939000881390008E3010008D6
:10007000E3010008E3010008E3010008E3010008D0
:10008000E3010008E3010008E3010008E3010008C0
:10009000E3010008E3010008E3010008A9390008B2
:1000A000E3010008E3010008E3010008E3010008A0
:1000B000E3010008E3010008E3010008E301000890
:1000C000E3010008E3010008E3010008E301000880
:1000D000E3010008E3010008E3010008E301000870
:1000E0000D3A0008E3010008E3010008E3010008FD
:1000F000E3010008E3010008E3010008E301000850
:10010000E3010008E3010008913A0008E301000858
:10011000E3010008E3010008E3010008E30100082F
:10012000E3010008E3010008E3010008E30100081F
:10013000E3010008E3010008E3010008E30100080F
:10014000E3010008E3010008E3010008DD2D0008D9
:10015000E3010008E3010008E30100087D3A00081C
:10016000E3010008E3010008E3010008E3010008DF
:10017000E3010008E3010008E3010008E3010008CF
:10018000E3010008E3010008E3010008E3010008BF
:10019000E3010008E3010008E3010008E3010008AF
:1001A000E3010008E3010008E3010008E30100089F
:1001B000E3010008E3010008E3010008E30100088F
:1001C000E3010008E3010008E3010008E30100087F
:1001D000E3010008E3010008E3010008E30100086F
:1001E00002E000F000F8FEE772B6374880F30888B6
:1001F000364880F3098836483649086040F20000E6
:10020000CCF200004EF63471CEF200010860BFF36C
:100210004F8FBFF36F8F40F20000C0F2F0004EF638
:100220008851CEF200010860BFF34F8FBFF36F8F8C
:100230004FF00000E1EE100A4EF63C71CEF20001E4
:100240000860062080F31488BFF36F8F02F08EFAE7
:1002500003F08EF94FF055301F491B4A91423CBFC5
:1002600041F8040BFAE71D49184A91423CBF41F896
:10027000040BFAE71A491B4A1B4B9A423EBF51F83E
:10028000040B42F8040BF8E700201849184A914281
:100290003CBF41F8040BFAE702F06CFA03F0BCF93A
:1002A000144C154DAC4203DA54F8041B8847F9E7A7
:1002B00000F042F8114C124DAC4203DA54F8041B22
:1002C0008847F9E702F054BA000600200022002017
:1002D0000000000808ED00E00000002000060020FB
:1002E000A03E0008002200204C22002050220020C6
:1002F000F0300020E0010008E0010008E001000803
:10030000E00100082DE9F04F2DED108AC1F80CD066
:10031000C3689D46BDEC108ABDE8F08F002383F3CF
:1003200011882846A047002001F0BAFDFEE701F041
:1003300023FD00DFFEE7000038B500F061FB02F0AE
:10034000E5F9054602F008FA0446D8B90F4B9D427C
:100350001AD001339D4218BF044641F2883504BFCC
:1003600001240025002002F0DBF90CB100F076F842
:1003700000F016FD00F0B0FB284600F0B7F800F0E2
:100380006DF8F9E70025EDE70546EBE7010007B05A
:1003900008B500F06DFBA0F120035842584108BD9C
:1003A00007B541F21203022101A8ADF8043000F0B4
:1003B0007DFB03B05DF804FB38B5302383F311886F
:1003C000174803680BB101F037FE164A14480023A2
:1003D0004FF47A7101F026FE002383F31188124C4A
:1003E000236813B12368013B2360636813B163681A
:1003F000013B63600D4D2B7833B963687BB90220F4
:1004000000F040FC322363602B78032B07D1636834
:100410002BB9022000F036FC4FF47A73636038BDCC
:1004200050220020B9030008702300206822002019
:10043000084B187003280CD8DFE800F00805020804
:10044000022000F00FBC022000F0FCBB024B002297
:100450005A60704768220020702300201F4B204AFA
:1004600010B51C461968013136D004339342F9D1D6
:100470006268A24230D31B4B9B6803F1006303F513
:1004800080439A4228D2002000F040FB0220FFF770
:10049000CFFF154B1A6C00221A64196E1A66196E7A
:1004A000596C5A64596E5A665A6E1A6942F0005273
:1004B0001A611A6922F000521A611B6972B64FF074
:1004C000E0233021C3F8084DD4E9003281F31188CC
:1004D0009D4683F30888104710BD00BF0040000808
:1004E0002040000800220020003802402DE9F04F93
:1004F00093B0AA4B00902022FF210AA89D6800F02B
:10050000F9FBA74A1378A3B9A6480121036011702B
:10051000302383F3118803680BB101F08DFDA24AEB
:10052000A04800234FF47A7101F07CFD002383F38F
:100530001188009B13B19D4B009A1A609C4A009C45
:100540001378032B1EBF00231370984A4FF0000A44
:1005500018BF5360D3465646D146012000F082FBB7
:1005600024B1924B1B68002B00F01182002000F098
:100570007FFA0390039B002BF2DB012000F062FB6B
:10058000039B213B162BE8D801A252F823F000BFB1
:10059000ED05000815060008A90600085B0500081F
:1005A0005B0500085B050008330700080309000825
:1005B0001D0800087F080008A7080008CD080008EB
:1005C0005B050008DF0800085B050008510900080A
:1005D0008D0600085B05000895090008F90500086C
:1005E0008D0600085B0500087F0800080220FFF761
:1005F000CFFE002840F0F581009B0221BAF1000FE8
:1006000008BF1C4605A841F21233ADF8143000F0C3
:100610004DFAA2E74FF47A7000F02AFA071EEBDBDE
:100620000220FFF7B5FE0028E6D0013F052F00F2BB
:10063000DA81DFE807F0030A0D101336052305936E
:10064000042105A800F032FA17E054480421F9E724
:1006500058480421F6E758480421F3E74FF01C08F6
:10066000404600F055FA08F104080590042105A859
:1006700000F01CFAB8F12C0FF2D1012000FA07F7B4
:1006800047EA0B0B5FFA8BFB4FF0000900F07EFB93
:1006900026B10BF00B030B2B08BF0024FFF780FEE5
:1006A0005BE746480421CDE7002EA5D00BF00B03F5
:1006B0000B2BA1D10220FFF76BFE074600289BD031
:1006C000012000F023FA0220FFF7B2FE00265FFAB5
:1006D00086F8404600F02AFA044690B100214046D0
:1006E00000F034FA01360028F1D1BA46044641F24E
:1006F0001213022105A8ADF814303E4600F0D6F9D9
:100700002BE70120FFF794FE2546244B9B68AB4264
:1007100007D9284600F0FCF9013040F06781043524
:10072000F3E7234B00251D70204BBA465D603E4623
:10073000ACE7002E3FF460AF0BF00B030B2B7FF404
:100740005BAF0220FFF774FE322000F091F9B0F1A8
:100750000008FFF651AF18F003077FF44DAF0F4AC2
:10076000926808EB050393423FF646AFB8F5807FE9
:100770003FF742AF124B0193B84523DD4FF47A7037
:1007800000F076F90390039A002AFFF635AF019B3B
:10079000039A03F8012B0137EDE700BF0022002088
:1007A0006C23002050220020B90300087023002091
:1007B0006822002004220020082200200C220020B1
:1007C0006C220020C820FFF7E3FD074600283FF415
:1007D00013AF1F2D11D8C5F1200242450AAB25F0F9
:1007E000030028BF424683490192184400F05CFA96
:1007F000019A8048FF2100F07DFA4FEAA8037D4965
:100800000193C8F38702284600F07CFA06460028C8
:100810003FF46DAF019B05EB830537E70220FFF73F
:10082000B7FD00283FF4E8AE00F0BCF900283FF423
:10083000E3AE0027B846704B9B68BB4218D91F2F08
:1008400011D80A9B01330ED027F0030312AA1344D8
:1008500053F8203C05934046042205A900F002FB12
:1008600004378046E7E7384600F052F90590F2E792
:10087000CDF81480042105A800F018F906E700233C
:10088000642104A8049300F007F900287FF4B4AEB3
:100890000220FFF77DFD00283FF4AEAE049800F083
:1008A00069F90590E6E70023642104A8049300F0A9
:1008B000F3F800287FF4A0AE0220FFF769FD0028BE
:1008C0003FF49AAE049800F065F9EAE70220FFF7DA
:1008D0005FFD00283FF490AE00F074F9E1E70220DC
:1008E000FFF756FD00283FF487AE05A9142000F05D
:1008F0006FF904210746049004A800F0D7F83946A0
:10090000B9E7322000F0B4F8071EFFF675AEBB075A
:100910007FF472AE384A926807EB090393423FF6C0
:100920006BAE0220FFF734FD00283FF465AE27F0E0
:1009300003074F44B9453FF4A9AE484600F0E8F834
:100940000421059005A800F0B1F809F10409F1E7C8
:100950004FF47A70FFF71CFD00283FF44DAE00F015
:1009600021F9002844D00A9B01330BD008220AA9A0
:10097000002000F0C7F900283AD02022FF210AA861
:1009800000F0B8F9FFF70CFD1C4801F08FFA13B026
:10099000BDE8F08F002E3FF42FAE0BF00B030B2BB6
:1009A0007FF42AAE0023642105A8059300F074F8B3
:1009B000074600287FF420AE0220FFF7E9FC8046BE
:1009C00000283FF419AEFFF7EBFC41F2883001F04C
:1009D0006DFA059800F024FA464600F0D7F93C4637
:1009E000BBE5064652E64FF0000905E6BA467EE64C
:1009F00037467CE66C22002000220020A086010001
:100A0000704700002DE9F84F4FF47A73DFF85880F3
:100A1000DFF8589006460D4602FB03F7002498F9CC
:100A200000305A1C5FFA84FA01D0A34212D159F85F
:100A3000240003682A46D3F820B031463B46D84705
:100A4000854207D1074B012083F800A0BDE8F88F4D
:100A50000124E4E7002CFBD04FF4FA7001F026FAF1
:100A60000020F3E7B82300201022002014220020E9
:100A700007B50023024601210DF107008DF807306C
:100A8000FFF7C0FF20B19DF8070003B05DF804FB3D
:100A90004FF0FF30F9E700000A4608B50421FFF7E0
:100AA000B1FF80F00100C0B2404208BD30B4074B36
:100AB0000A461978064B53F821402368DD69054B37
:100AC0000146AC46204630BC604700BFB82300203A
:100AD00014220020A086010070B501F009FD094E26
:100AE000094D3080002428683388834208D901F0FA
:100AF000F9FC2B6804440133B4F5804F2B60F2D32A
:100B000070BD00BFBA2300207823002001F0B2BDE1
:100B100000F1006000F580400068704700F100605F
:100B2000920000F5804001F031BD0000054B1A68CD
:100B3000054B1B889B1A834202D9104401F0D2BC9A
:100B40000020704778230020BA23002038B5084DD4
:100B5000044629B128682044BDE8384001F0E2BCD1
:100B60002868204401F0C6FC0028F3D038BD00BF3F
:100B70007823002010F003030AD1B0F5047F05D2DA
:100B800000F10050A0F51040D0F80038184670472A
:100B90000023FBE700F10050A0F51040D0F8100A48
:100BA00070470000064991F8243033B10023086AE9
:100BB00081F824300822FFF7B1BF0120704700BF41
:100BC0007C230020014B1868704700BF002004E020
:100BD00070B5194B1D68194B0138C5F30B04084457
:100BE0002D0C04221E88A6420BD15C680A46013CEB
:100BF000824213460FD214F9016F4EB102F8016B15
:100C0000F6E7013A03F10803ECD181420B4602D228
:100C10002C2203F8012B0A4A05241688AE4204D17F
:100C2000984284BF967803F8016B013C02F10402FC
:100C3000F3D1581A70BD00BF002004E0803B0008CB
:100C40006C3B0008022804D1054B4FF400429A6126
:100C500070470128FCD1024B4FF48052F7E700BFE8
:100C600000100240022804D1054B4FF000429A6167
:100C700070470128FCD1024B4FF08052F7E700BFCC
:100C800000100240022805D1064A536983F400434C
:100C9000536170470128FCD1024A536983F48053A1
:100CA000F6E700BF0010024010B50023934203D0C6
:100CB000CC5CC4540133F9E710BD000010B5013815
:100CC00010F9013F3BB191F900409C4203D11AB1A8
:100CD0000131013AF4E71AB191F90020981A10BDD8
:100CE0001046FCE703460246D01A12F9011B002900
:100CF000FAD1704702440346934202D003F8011B25
:100D0000FAE770472DE9F8431F4D144695F8242063
:100D10000746884652BBDFF870909CB395F82430A4
:100D20002BB92022FF2148462F62FFF7E3FF95F8F9
:100D30002400C0F10802A24228BF2246D6B2414692
:100D4000920005EB8000FFF7AFFF95F82430A41B5D
:100D50001E44F6B2082E17449044E4B285F824608D
:100D6000DBD1FFF71FFF0028D7D108E02B6A03EB88
:100D700082038342CFD0FFF715FF0028CBD100209C
:100D8000BDE8F8830120FBE77C230020024B1A78A2
:100D9000024B1A70704700BFB823002010220020B9
:100DA00038B5194C194D204600F0C0FB29462046A5
:100DB00000F0E8FB2D6816486A6DD2F8043843F05D
:100DC0000203C2F8043801F071F81249284600F015
:100DD000DFFC6A6D104DD2F8043828680F4923F003
:100DE0000203C2F80438A0424FF4E1330B6001D093
:100DF00000F0FCFA6868A04204D0BDE8384007491A
:100E000000F0F4BA38BD00BF98280020883C0008E4
:100E100040420F00903C000814220020A423002030
:100E200070B50C4B0C4D1E780C4B55F826209A4291
:100E300004460DD00A4B002114221846FFF75AFF32
:100E40000460014655F82600BDE8704000F0CEBAB7
:100E500070BD00BFB8230020142200209828002075
:100E6000A423002030B5094D0A4491420DD011F859
:100E7000013B5840082340F30004013B2C4013F091
:100E8000FF0384EA5000F6D1EFE730BD2083B8EDD0
:100E9000026843681143016003B1184770470000BE
:100EA000024AD36843F0C003D36070470014014086
:100EB00010B5084C084A0021204600F075FA074B8F
:100EC000C4F85C3203F1454303F52943C4F86032AA
:100ED00010BD00BFBC230020A10E0008001401407B
:100EE000234A037C002918BF0A46012B30B5C0F8FD
:100EF00068220CD11F4B984209D11F4B596C41F00D
:100F000020015964596E41F0200159665B6EB2F9B7
:100F100004501468D0F86032D0F85C12002D03EB56
:100F20005403B3FBF4F3BEBF23F0070503F007033C
:100F300043EA450394888B60D38843F040030B61F8
:100F4000138943F001034B6144F4045343F02C0331
:100F5000CB6004F4A05400230B60B4F5806F0B68E1
:100F60004B680CBF7F23FF2380F8643230BD00BF85
:100F7000A03B0008BC230020003802402DE9F041CE
:100F8000D0F85C62F7683368DA0504469DB20DD587
:100F9000302383F311884FF480610430FFF778FF2A
:100FA0006FF480733360002383F31188302383F35D
:100FB000118804F1040815F02F033AD183F3118846
:100FC000380615D5290613D5302383F3118804F18B
:100FD000380000F065F900284EDA0821201DFFF7DF
:100FE00057FF4FF67F733B40F360002383F3118874
:100FF0007A0616D56B0614D5302383F31188D4E90D
:1010000013239A420AD1236C43B127F040073F04CF
:101010001021201D3F0CFFF73BFFF760002383F3F7
:101020001188D4F86822D36843B3BDE8F041106951
:1010300018472B0714D015F0080F0CBF00214FF4F0
:101040008071E80748BF41F02001AA0748BF41F07E
:1010500040016B0748BF41F080014046FFF718FF91
:10106000AD06736805D594F864122046194000F067
:10107000CBF93568ADB29EE77060B6E7BDE8F081A8
:10108000F8B5154682680669AA420B46816938BFE1
:101090008568761AB54204460BD218462A46FFF7F1
:1010A00003FEA3692B44A361A3685B1BA3602846CE
:1010B000F8BD0CD918463246FFF7F6FDAF1BE168C4
:1010C0003A463044FFF7F0FDE3683B44EBE718464F
:1010D0002A46FFF7E9FDE368E5E7000083689342ED
:1010E000F7B51546044638BF8568D0E90460361A5E
:1010F000B5420BD22A46FFF7D7FD63692B446361E3
:10110000A36828465B1BA36003B0F0BD0DD932462F
:101110000191FFF7C9FD0199E068AF1B3A463144E0
:10112000FFF7C2FDE3683B44E9E72A46FFF7BCFD51
:10113000E368E4E710B50A440024C361029B8460BD
:10114000C0E90000C0E90511C1600261036210BD81
:1011500008B5D0E90532934201D1826882B982682C
:10116000013282605A1C42611970D0E904329A42FD
:1011700024BFC3684361002100F0B4FE002008BD15
:101180004FF0FF30FBE7000070B5302304460E46F9
:1011900083F31188A568A5B1A368A269013BA36088
:1011A000531CA36115782269934224BFE368A361AD
:1011B000E3690BB120469847002383F31188284642
:1011C00007E03146204600F07DFE0028E2DA85F394
:1011D000118870BD2DE9F74F04460E461746984614
:1011E000D0F81C904FF0300A8AF311884FF0000BB2
:1011F000154665B12A4631462046FFF741FF0346B2
:1012000060B94146204600F05DFE0028F1D0002381
:1012100083F31188781B03B0BDE8F08FB9F1000F9C
:1012200003D001902046C847019B8BF31188ED1A2B
:101230001E448AF31188DCE7C0E90511C160C3616F
:101240001144009B8260C0E90000016103627047A5
:10125000F8B504460D461646302383F31188A76877
:10126000A7B1A368013BA36063695A1C62611D704A
:10127000D4E904329A4224BFE3686361E3690BB1A5
:1012800020469847002080F3118807E03146204629
:1012900000F018FE0028E2DA87F31188F8BD00009C
:1012A000D0E905239A4210B501D182687AB98268E3
:1012B000013282605A1C82611C7803699A4224BF01
:1012C000C3688361002100F00DFE204610BD4FF081
:1012D000FF30FBE72DE9F74F04460E4617469846C8
:1012E000D0F81C904FF0300A8AF311884FF0000BB1
:1012F000154665B12A4631462046FFF7EFFE034604
:1013000060B94146204600F0DDFD0028F1D0002301
:1013100083F31188781B03B0BDE8F08FB9F1000F9B
:1013200003D001902046C847019B8BF31188ED1A2A
:101330001E448AF31188DCE70268436811430160A8
:1013400003B11847704700001430FFF743BF000097
:101350004FF0FF331430FFF73DBF00003830FFF788
:10136000B9BF00004FF0FF333830FFF7B3BF0000C4
:101370001430FFF709BF00004FF0FF311430FFF7C2
:1013800003BF00003830FFF763BF00004FF0FF32AB
:101390003830FFF75DBF0000012914BF6FF0130064
:1013A00000207047FFF784BD37B515460E4A02602E
:1013B00000224260C0E902220122044602740B4668
:1013C000009000F15C014FF480721430FFF7B2FE20
:1013D00000942B464FF4807204F5AE7104F138008E
:1013E000FFF72AFF03B030BDB43B000810B530232F
:1013F000044683F31188FFF773FD02232374002052
:1014000080F3118810BD000038B5C36904460D464D
:101410001BB904210844FFF78FFF294604F114008B
:10142000FFF796FE002806DA201D4FF40061BDE8A4
:101430003840FFF781BF38BD02684368114301603F
:1014400003B118477047000013B5446BD4F89434C7
:101450001A681178042915D1217C022912D1197931
:10146000128901238B4013420CD101A904F14C00D5
:1014700001F034FFD4F89444019B2179024620689E
:1014800000F0D0F902B010BD143001F0B7BE00007A
:101490004FF0FF33143001F0B1BE00004C3001F0CA
:1014A00089BF00004FF0FF334C3001F083BF0000D4
:1014B000143001F085BE00004FF0FF31143001F010
:1014C0007FBE00004C3001F055BF00004FF0FF32EE
:1014D0004C3001F04FBF00000020704710B5D0F82D
:1014E00094341A6811780429044617D1017C022922
:1014F00014D15979528901238B4013420ED11430F3
:1015000001F018FE024648B1D4F894444FF48073B9
:1015100061792068BDE8104000F072B910BD00008C
:10152000406BFFF7DBBF0000704700007FB5124B38
:10153000036000234360C0E90233012502260F4BFC
:10154000057404460290019300F184022946009636
:101550004FF48073143001F0C9FD094B0294CDE9BA
:10156000006304F523724FF48073294604F14C00A4
:1015700001F090FE04B070BDDC3B000821150008AE
:10158000491400080B68302282F311880A7903EBB2
:10159000820290614A79093243F822008A7912B1B5
:1015A00003EB820398610223C0F8941403740020B3
:1015B00080F311887047000038B5037F044613B1EB
:1015C00090F85430ABB9201D01250221FFF734FFFC
:1015D00004F1140025776FF0010100F08FFC84F80E
:1015E000545004F14C006FF00101BDE8384000F0A8
:1015F00085BC38BD10B5012104460430FFF71CFF3F
:101600000023237784F8543010BD000038B5044619
:101610000025143001F082FD04F14C00257701F023
:1016200051FE201D84F854500121FFF705FF20468C
:10163000BDE83840FFF752BF90F8443003F0600334
:10164000202B07D190F84520212A4FF0000303D822
:101650001F2A06D800207047222AFBD1C0E90E338A
:1016600003E0034A82630722C263036401207047D8
:101670001C22002037B5D0F894341A681178042958
:1016800004461AD1017C022917D119791289012344
:101690008B40134211D100F14C05284601F0D2FED7
:1016A00058B101A9284601F019FED4F89444019BD1
:1016B00021790246206800F0B5F803B030BD000083
:1016C000F0B500EB810385B09E6904460D46FEB17E
:1016D000302383F3118804EB8507301D0821FFF7C1
:1016E000ABFEFB685B691B6806F14C001BB1019007
:1016F00001F002FE019803A901F0F0FD024648B195
:10170000039B2946204600F08DF8002383F31188BF
:1017100005B0F0BDFB685A691268002AF5D01B8A33
:10172000013B1340F1D104F14402EAE7093138B535
:1017300050F82140DCB1302383F31188D4F894248D
:101740001368527903EB8203DB689B695D6845B1DE
:1017500004216018FFF770FE294604F1140001F01F
:10176000F3FC2046FFF7BAFE002383F3118838BD4F
:101770007047000001F052B8012303700023C0E954
:101780000133C36183620362C362436203637047D0
:1017900038B50446302383F311880025C0E903558A
:1017A000C0E90555416001F049F80223237085F333
:1017B0001188284638BD000070B500EB810305464E
:1017C0005069DA600E46144618B110220021FFF766
:1017D00091FAA06918B110220021FFF78BFA314667
:1017E0002846BDE8704001F0F3B80000826802F0BE
:1017F000011282600022C0E90422826101F074B902
:10180000F0B400EB81044789E4680125A4698D40A8
:101810003D43458123600023A2606360F0BC01F07A
:101820008FB90000F0B400EB81040789E46801255A
:1018300064698D403D43058123600023A26063609D
:10184000F0BC01F009BA000070B50223002504467F
:101850000370C0E90255C0E90455C564856180F88C
:10186000345001F051F863681B6823B129462046C3
:10187000BDE87040184770BD0378052B10B50446CD
:101880000AD080F850300523037043681B680BB101
:10189000042198470023A36010BD000001780529AA
:1018A00006D190F85020436802701B6803B11847B6
:1018B0007047000070B590F83430044613B100232F
:1018C00080F8343004F14402204601F02FF96368B7
:1018D0009B68B3B994F8443013F0600535D000210B
:1018E000204601F0CFFB0021204601F0C1FB6368D8
:1018F0001B6813B1062120469847062384F834302C
:1019000070BD204698470028E4D0B4F84A30E26B16
:101910009A4288BFE36394F94430E56B002B4FF0A3
:10192000300380F20381002D00F0F280092284F858
:10193000342083F311880021D4E90E232046FFF7D9
:1019400071FF002383F31188DAE794F8452003F050
:101950007F0343EA022340F20232934200F0C58043
:1019600021D8B3F5807F48D00DD8012B3FD0022B72
:1019700000F09380002BB2D104F14C02A26302224A
:10198000E2632364C1E7B3F5817F00F09B80B3F588
:10199000407FA4D194F84630012BA0D1B4F84C304C
:1019A00043F0020332E0B3F5006F4DD017D8B3F522
:1019B000A06F31D0A3F5C063012B90D8636894F871
:1019C00046205E6894F84710B4F848302046B04787
:1019D000002884D04368A3630368E3631AE0B3F587
:1019E000106F36D040F6024293427FF478AF5C4BE2
:1019F000A3630223E3630023C3E794F84630012B7B
:101A00007FF46DAFB4F84C3023F00203C4E90E55F7
:101A1000A4F84C30256478E7B4F84430B3F5A06FEF
:101A20000ED194F8463084F84E30204600F0C4FFC2
:101A300063681B6813B10121204698470323237074
:101A40000023C4E90E339CE704F14F03A363012391
:101A5000C3E72378042B10D1302383F31188204669
:101A6000FFF7C4FE85F311880321636884F84F50A3
:101A700021701B680BB12046984794F84630002B24
:101A8000DED084F84F300423237063681B68002B7A
:101A9000D6D0022120469847D2E794F848301D0658
:101AA00003F00F0120460AD501F032F8012804D0D6
:101AB00002287FF414AF2B4B9AE72B4B98E701F0E9
:101AC00019F8F3E794F84630002B7FF408AF94F848
:101AD000483013F00F01B3D01A06204602D501F0AA
:101AE000E5FAADE701F0D8FAAAE794F84630002B02
:101AF0007FF4F5AE94F8483013F00F01A0D01B0628
:101B0000204602D501F0BEFA9AE701F0B1FA97E754
:101B1000142284F8342083F311882B462A46294660
:101B20002046FFF76DFE85F31188E9E65DB11522C9
:101B300084F8342083F311880021D4E90E23204651
:101B4000FFF75EFEFDE60B2284F8342083F3118854
:101B50002B462A4629462046FFF764FEE3E700BFEE
:101B60000C3C0008043C0008083C000838B590F81C
:101B700034300446002B3ED0063BDAB20F2A34D86C
:101B80000F2B32D8DFE803F0373131082232313100
:101B90003131313131313737C56BB0F84A309D4280
:101BA00014D2C3681B8AB5FBF3F203FB12556DB95F
:101BB000302383F311882B462A462946FFF732FE4D
:101BC00085F311880A2384F834300EE0142384F856
:101BD0003430302383F3118800231A4619462046F7
:101BE000FFF70EFE002383F3118838BD036C03B1A9
:101BF00098470023E7E70021204601F043FA00213F
:101C0000204601F035FA63681B6813B106212046AF
:101C100098470623D7E7000010B590F83430142B0E
:101C2000044629D017D8062B05D001D81BB110BD0A
:101C3000093B022BFBD80021204601F023FA0021AA
:101C4000204601F015FA63681B6813B1062120468F
:101C50009847062319E0152BE9D10B2380F834307F
:101C6000302383F3118800231A461946FFF7DAFD63
:101C7000002383F31188DAE7C3689B695B68002B54
:101C8000D5D1036C03B19847002384F83430CEE7F4
:101C900000230375826803691B6899689142FBD22F
:101CA0005A680360426010605860704700230375F3
:101CB000826803691B6899689142FBD85A6803607F
:101CC000426010605860704708B50846302383F3BF
:101CD00011880B7D032B05D0042B0DD02BB983F37A
:101CE000118808BD8B6900221A604FF0FF338361B1
:101CF000FFF7CEFF0023F2E7D1E9003213605A600C
:101D0000F3E70000FFF7C4BF054BD96808751868F2
:101D100002681A60536001220275D860FEF7F2BAB9
:101D20002826002030B50C4BDD684B1C87B00446DC
:101D30000FD02B46094A684600F074F92046FFF799
:101D4000E3FF009B13B1684600F076F9A86907B07D
:101D500030BDFFF7D9FFF9E728260020C91C00088D
:101D6000044B1A68DB6890689B68984294BF002017
:101D70000120704728260020084B10B51C68D86841
:101D800022681A60536001222275DC60FFF78EFF23
:101D900001462046BDE81040FEF7B4BA28260020D0
:101DA000044B1A68DB6892689B689A4201D9FFF776
:101DB000E3BF70472826002038B5074C074908487C
:101DC000012300252370656001F07AFB0223237054
:101DD00085F3118838BD00BF90280020143C00080E
:101DE0002826002000F05EB9EFF3118020B9EFF350
:101DF0000583302282F311887047000010B530B996
:101E0000EFF30584C4F3080414B180F3118810BD06
:101E1000FFF7C6FF84F31188F9E70000034A516811
:101E200053685B1A9842FBD8704700BF001000E06F
:101E30008B60022308618B82084670478368A3F198
:101E4000840243F8142C026943F8442C426943F895
:101E5000402C094A43F8242CC26843F8182C02226B
:101E600003F80C2C002203F80B2C044A43F8102C26
:101E7000A3F12000704700BF1D03000828260020A2
:101E800008B5FFF7DBFFBDE80840FFF73BBF0000E8
:101E9000024BDB6898610F20FFF736BF2826002031
:101EA000302383F31188FFF7F3BF000008B5014624
:101EB000302383F311880820FFF734FF002383F3D6
:101EC000118808BD064BDB6839B1426818605A605A
:101ED000136043600420FFF725BF4FF0FF307047C9
:101EE000282600200368984206D01A6802605060D5
:101EF00099611846FFF706BF7047000038B50446E1
:101F00000D462068844200D138BD036823605C60C0
:101F10008561FFF7F7FEF4E710B503689C68A242FD
:101F20000CD85C688A600B604C60216059609968CD
:101F30008A1A9A604FF0FF33836010BD1B68121B32
:101F4000ECE700000A2938BF0A2170B504460D46A7
:101F50000A26601901F0ACFA01F094FA041BA542BC
:101F600003D8751C2E460446F3E70A2E04D9BDE8B3
:101F70007040012001F0E4BA70BD0000F8B5144BC8
:101F80000D46D96103F1100141600A2A1969826086
:101F900038BF0A22016048601861A818144601F091
:101FA00077FA0A2701F06EFA431BA342064606D3CE
:101FB0007C1C281901F07CFA27463546F2E70A2FE7
:101FC00004D9BDE8F840012001F0BABAF8BD00BF5D
:101FD00028260020F8B506460D4601F053FA0F4AB0
:101FE000134653F8107F9F4206D12A4601463046D9
:101FF000BDE8F840FFF7C2BFD169BB68441A2C198D
:1020000028BF2C46A34202D92946FFF79BFF224650
:1020100031460348BDE8F840FFF77EBF2826002080
:102020003826002010B4C0E9032300235DF8044BD8
:102030004361FFF7CFBF000010B5194C23699842E8
:102040000DD0D0E90032816813605A609A680A4462
:102050009A60002303604FF0FF33A36110BD234655
:10206000026843F8102F53600022026022699A42EE
:1020700003D1BDE8104001F015BA936881680B44A4
:10208000936001F0FFF92269E1699268441AA24263
:10209000E4D91144BDE81040091AFFF753BF00BF4F
:1020A000282600202DE9F047DFF8BC8008F1100752
:1020B0002C4ED8F8105001F0E5F9D8F81C40AA6869
:1020C000031B9A423ED81444D5E900324FF0000970
:1020D000C8F81C4013605A60C5F80090D8F810305A
:1020E000B34201D101F0DEF989F31188D5E903315A
:1020F00028469847302383F311886B69002BD8D08A
:1021000001F0C0F96A69A0EB04094A4582460DD284
:10211000022001F015FA0022D8F81030B34208D19D
:1021200051462846BDE8F047FFF728BF121A22445F
:10213000F2E712EB090938BF4A4629463846FFF74D
:10214000EBFEB5E7D8F81030B34208D01444211A9A
:10215000C8F81C00A960BDE8F047FFF7F3BEBDE872
:10216000F08700BF38260020282600200020704776
:10217000FEE70000704700004FF0FF30704700009E
:1021800002290CD0032904D00129074818BF0020D8
:102190007047032A05D8054800EBC2007047044881
:1021A00070470020704700BFEC3C00082C22002044
:1021B000A03C000870B59AB00546084601A914462F
:1021C00000F0C2F801A8FEF78DFD431C5B00C5E9D5
:1021D00000340022237003236370C6B201AB0234C3
:1021E0001046D1B28E4204F1020401D81AB070BD7B
:1021F00013F8011B04F8021C04F8010C0132F0E78B
:1022000008B5302383F311880348FFF733FA00231E
:1022100083F3118808BD00BF9828002090F844304F
:1022200003F01F02012A07D190F845200B2A03D1A1
:102230000023C0E90E3315E003F06003202B08D122
:10224000B0F848302BB990F84520212A03D81F2A2E
:1022500004D8FFF7F1B9222AEBD0FAE7034A8263E8
:102260000722C26303640120704700BF23220020BD
:1022700007B5052917D8DFE801F019160319192049
:10228000302383F31188104A01900121FFF794FA5B
:1022900001980E4A0221FFF78FFA0D48FFF7B6F9B1
:1022A000002383F3118803B05DF804FB302383F32C
:1022B00011880748FFF780F9F2E7302383F311888C
:1022C0000348FFF797F9EBE7403C0008643C00083F
:1022D0009828002038B50C4D0C4C0D492A4604F1C5
:1022E0000800FFF767FF05F1CA0204F11000094971
:1022F000FFF760FF05F5CA7204F118000649BDE852
:102300003840FFF757BF00BF602D00202C2200206F
:10231000203C00082A3C0008353C000870B5044603
:1023200008460D46FEF7DEFCC6B2204601340378AF
:102330000BB9184670BD32462946FEF7BFFC00288F
:10234000F3D10120F6E700002DE9F04705460C46E1
:10235000FEF7C8FC2C49C6B22846FFF7DFFF08B1DC
:102360000836F6B229492846FFF7D8FF08B11036DB
:10237000F6B2632E0BD8DFF89080DFF89090244FF0
:10238000DFF898A02E7846B92670BDE8F087294678
:102390002046BDE8F04701F0CBBB252E30D1072207
:1023A00041462846FEF78AFC80B91A4B224603F1C3
:1023B0000C0153F8040B42F8040B8B42F9D1198835
:1023C0009B781180937007350F34DBE7082249466C
:1023D0002846FEF773FC98B90F4BA21C197809091F
:1023E0000232C95D02F8041C13F8011B01F00F0151
:1023F0005345C95D02F8031CF0D118340835C1E714
:1024000004F8016B0135BDE70C3D0008353C0008C0
:10241000243D0008143D0008107AFF1F1C7AFF1F9E
:10242000BFF34F8F024AD368DB03FCD4704700BF71
:10243000003C024008B5094B1B7873B9FFF7F0FF69
:10244000074B1A69002ABFBF064A5A6002F1883258
:102450005A601A6822F480621A6008BDBE2F0020FC
:10246000003C02402301674508B50B4B1B7893B92C
:10247000FFF7D6FF094B1A6942F000421A611A6849
:1024800042F480521A601A6822F480521A601A6864
:1024900042F480621A6008BDBE2F0020003C02405A
:1024A0000B28F0B516D80C4C0C4923787BB90C4D91
:1024B0000E460C234FF0006255F8047B46F8042BBF
:1024C000013B13F0FF033A44F6D10123237051F886
:1024D0002000F0BD0020FCE7F02F0020C02F0020DE
:1024E000383D0008014B53F820007047383D000884
:1024F0000C2070470B2810B5044601D9002010BDF0
:10250000FFF7CEFF064B53F824301844C21A0BB91C
:102510000120F4E712680132F0D1043BF6E700BF76
:10252000383D00080B2838B5044628D8FFF75CFC76
:10253000FFF776FFFFF77EFF124AF323D360E30035
:10254000DBB243F4007343F002031361136943F4F5
:102550008033136105462046FFF762FFFFF7A0FFB7
:10256000094B53F8241000F0E9F82846FFF77CFFE8
:10257000FFF744FC2046BDE83840FFF7BBBF002012
:1025800038BD00BF003C0240383D000812F0010396
:102590002DE9F04105460E4614464BD18218B2F1A2
:1025A000016F61D8314B1B6813F001035CD0304FD1
:1025B000FFF71AFCFFF73EFFF323FB60FFF730FF46
:1025C000314640F20128032C18D824F00104284E8B
:1025D0000C446D1A40F20118A142336905EB010762
:1025E0002AD123F001033361FFF73EFFFFF706FC1A
:1025F0000120BDE8F081043C0435E4E7AB07E4D1F9
:102600003B6923F440733B613B6943EA08033B6148
:1026100051F8046B2E60BFF34F8FFFF701FF2B685B
:102620009E42E8D03B6923F001033B61FFF71CFFAA
:10263000FFF7E4FB0020DCE723F4407333613369E8
:1026400043EA080333610B883B80BFF34F8FFFF7EA
:10265000E7FE3F8831F8023BBFB2BB42BCD03369D2
:1026600023F001033361E1E71846C2E70038024076
:10267000003C0240084908B50B7828B11BB9FFF7A8
:10268000D9FE01230B7008BD002BFCD0BDE808402B
:102690000870FFF7E9BE00BFBE2F002010B502444E
:1026A000064BD2B2904200D110BD441C00B253F888
:1026B000200041F8040BE0B2F4E700BF50280040CE
:1026C0000F4B30B51C6F240407D41C6F44F4007406
:1026D0001C671C6F44F400441C670A4C236843F4D5
:1026E000807323600244084BD2B2904200D130BDC7
:1026F000441C00B251F8045B43F82050E0B2F4E708
:1027000000380240007000405028004007B5012208
:1027100001A90020FFF7C2FF019803B05DF804FB98
:1027200013B50446FFF7F2FFA04205D0012201A92C
:1027300000200194FFF7C4FF02B010BD70470000F5
:10274000034B1A681AB9034AD2F874281A60704702
:10275000F42F00200030024008B5FFF7F1FF024BD4
:102760001868C0F3407008BDF42F002070470000C7
:10277000FEE700000A4B0B480B4A90420BD30B4B71
:10278000DA1C121AC11E22F003028B4238BF00224B
:102790000021FEF7AFBA53F8041B40F8041BECE726
:1027A000EC3E0008F0300020F0300020F030002037
:1027B00070B5D0E915439E6800224FF0FF3504EB59
:1027C00042135101D3F800090028BEBFD3F8000915
:1027D00040F08040C3F80009D3F8000B0028BEBFCA
:1027E000D3F8000B40F08040C3F8000B01326318AF
:1027F0009642C3F80859C3F8085BE0D24FF00113C2
:10280000C4F81C3870BD0000890141F0200101614D
:1028100003699B06FCD41220FFF700BB10B5054CE2
:102820002046FEF7A9FF4FF0A0436365024BA36566
:1028300010BD00BFF82F00208C3D000870B5037854
:10284000012B054650D12A4B446D98421BD1294B90
:102850005A6B42F080025A635A6D42F080025A6508
:102860005A6D5A6942F080025A615A6922F0800218
:102870005A610E2143205B6900F022FC1E4BE3608D
:102880001E4BC4F800380023C4F8003EC023236068
:102890006E6D4FF40413A3633369002BFCDA01233C
:1028A00033610C20FFF7BAFA3369DB07FCD412203E
:1028B000FFF7B4FA3369002BFCDA0026A66028463D
:1028C000FFF776FF6B68C4F81068DB68C4F814681B
:1028D000C4F81C684BB90A4BA3614FF0FF33636126
:1028E000A36843F00103A36070BD064BF4E700BF8B
:1028F000F82F00200038024040140040030020025E
:10290000003C30C0083C30C0F8B5446D054600219D
:102910002046FFF779FFA96D00234FF001128F6861
:10292000C4F834384FF00066C4F81C284FF0FF306C
:1029300004EB431201339F42C2F80069C2F8006BF6
:10294000C2F80809C2F8080BF2D20B686A6DEB6591
:10295000636210231361166916F01006FBD1122072
:10296000FFF75CFAD4F8003823F4FE63C4F80038AB
:10297000A36943F4402343F01003A3610923C4F87F
:102980001038C4F814380A4BEB604FF0C043C4F859
:10299000103B084BC4F8003BC4F81069C4F8003978
:1029A000EB6D03F1100243F48013EA65A362F8BDF6
:1029B000683D000840800010426D90F84E10D2F83B
:1029C000003823F4FE6343EA0113C2F8003870476D
:1029D0002DE9F84300EB8103456DDA68166806F0CF
:1029E0000306731E022B05EB41130C4680460FFABB
:1029F00081F94FEA41104FF00001C3F8101B4FF06E
:102A0000010104F1100398BFB60401FA03F39169C0
:102A10008EBF334E06F1805606F5004600293AD0A7
:102A2000578A04F15801490137436F50D5F81C18F3
:102A30000B43C5F81C382B180021C3F81019536933
:102A40000127611EA7409BB3138A928B9B08012A22
:102A500088BF5343D8F85C20981842EA034301F139
:102A6000400205EB8202C8F85C002146536028460C
:102A7000FFF7CAFE08EB8900C3681B8A43EA845348
:102A8000483464011E432E51D5F81C381F43C5F845
:102A90001C78BDE8F88305EB4917D7F8001B21F433
:102AA0000041C7F8001BD5F81C1821EA0303C0E752
:102AB00004F13F0305EB83030A4A5A602846214686
:102AC000FFF7A2FE05EB4910D0F8003923F40043CC
:102AD000C0F80039D5F81C3823EA0707D7E700BF4C
:102AE0000080001000040002826D1268C265FFF7CA
:102AF0005FBE00005831436D49015B5813F400403C
:102B000004D013F4001F0CBF022001207047000006
:102B10004831436D49015B5813F4004004D013F46D
:102B2000001F0CBF022001207047000000EB810154
:102B3000CB68196A0B6813604B68536070470000DC
:102B400000EB810330B5DD68AA691368D36019B959
:102B5000402B84BF402313606B8A1468426D1C4471
:102B6000013CB4FBF3F46343033323F0030302EBB0
:102B7000411043EAC44343F0C043C0F8103B2B6804
:102B800003F00303012B09B20ED1D2F8083802EB8F
:102B9000411013F4807FD0F8003B14BF43F0805302
:102BA00043F00053C0F8003B02EB4112D2F8003B67
:102BB00043F00443C2F8003B30BD00002DE9F04172
:102BC000244D6E6D06EB40130446D3F8087BC3F822
:102BD000087B38070AD5D6F81438190706D505EB4F
:102BE00084032146DB6828465B689847FA071FD5AF
:102BF000D6F81438DB071BD505EB8403D968CCB9AC
:102C00008B69488A5A68B2FBF0F600FB16228AB933
:102C10001868DA6890420DD2121AC3E900243023F2
:102C200083F311880B482146FFF78AFF84F311884C
:102C3000BDE8F081012303FA04F26B8923EA020361
:102C40006B81CB68002BF3D021460248BDE8F041F0
:102C5000184700BFF82F002000EB810370B5DD6836
:102C6000436D6C692668E6604A0156BB1A444FF40E
:102C70000020C2F810092A6802F00302012A0AB2F1
:102C80000ED1D3F8080803EB421410F4807FD4F877
:102C9000000914BF40F0805040F00050C4F8000913
:102CA00003EB4212D2F8000940F00440C2F80009D8
:102CB000D3F83408012202FA01F10143C3F83418B1
:102CC00070BD19B9402E84BF4020206020682E8A34
:102CD0008419013CB4FBF6F440EAC44040F00050D3
:102CE0001A44C6E72DE9F8433B4D6E6D06EB4013E1
:102CF0000446D3F80889C3F8088918F0010F4FEA91
:102D000040171AD0D6F81038DB0716D505EB80032C
:102D1000D9684B691868DA68904230D2121A4FF0BD
:102D200000091A60C3F80490302383F31188214608
:102D30002846FFF791FF89F3118818F0800F1CD007
:102D4000D6F834380126A640334216D005EB84036A
:102D50006D6DD3F80CC0DCF814200134E4B2D2F865
:102D600000E005EB04342F445168714515D3D5F8C4
:102D7000343823EA0606C5F83468BDE8F883012331
:102D800003FA04F22B8923EA02032B818B68002BC0
:102D9000D3D0214628469847CFE7BCF81000AEEBC9
:102DA0000103834228BF0346D7F8180980B2B3EB6A
:102DB000800FE2D89068A0F1040959F8048FC4F894
:102DC0000080A0EB09089844B8F1040FF5D8184426
:102DD0000B4490605360C7E7F82F00202DE9F74FB0
:102DE000A24C656D6E69AB691E4016F480586E6129
:102DF00007D02046FEF728FD03B0BDE8F04F00F0F5
:102E00004DBC002E12DAD5F8003E98489B071EBF35
:102E1000D5F8003E23F00303C5F8003ED5F804388A
:102E200023F00103C5F80438FEF738FD370505D552
:102E30008E48FFF7BDFC8D48FEF71EFDB0040CD593
:102E4000D5F8083813F0060FEB6823F470530CBF65
:102E500043F4105343F4A053EB6031071BD5636870
:102E6000DB681BB9AB6923F00803AB612378052B42
:102E70000CD1D5F8003E7D489A071EBFD5F8003E1C
:102E800023F00303C5F8003EFEF708FD6368DB6826
:102E90000BB176489847F30274D4B70227D5D4F81B
:102EA0005490DFF8C8B100274FF0010A09EB471230
:102EB000D2F8003B03F44023B3F5802F11D1D2F8B0
:102EC000003B002B0DDA62890AFA07F322EA0303BA
:102ED000638104EB8703DB68DB6813B1394658462E
:102EE0009847A36D01379B68FFB29F42DED9F00679
:102EF00017D5676D3A6AC2F30A1002F00F0302F4A5
:102F0000F012B2F5802F00F08580B2F5402F08D185
:102F100004EB83030022DB681B6A07F580579042AD
:102F20006AD13003D5F8184813D5E10302D5002043
:102F3000FFF744FEA20302D50120FFF73FFE630323
:102F400002D50220FFF73AFE270302D50320FFF740
:102F500035FE75037FF550AFE00702D50020FFF77F
:102F6000C1FEA10702D50120FFF7BCFE620702D512
:102F70000220FFF7B7FE23077FF53EAF0320FFF7E0
:102F8000B1FE39E7636DDFF8E4A0019300274FF04D
:102F90000109A36D9B685FFA87FB9B453FF67DAFF8
:102FA000019B03EB4B13D3F8001901F44021B1F559
:102FB000802F1FD1D3F8001900291BDAD3F800198C
:102FC00041F09041C3F80019D3F800190029FBDB48
:102FD0005946606DFFF718FC218909FA0BF321EAC5
:102FE0000303238104EB8B03DB689B6813B1594611
:102FF000504698470137CCE7910708BFD7F80080C3
:10300000072A98BF03F8018B02F1010298BF4FEA2B
:10301000182884E7023304EB830207F580575268CF
:10302000D2F818C0DCF80820DCE9001CA1EB0C0C7D
:10303000002188420AD104EB830463689B699A6883
:1030400002449A605A6802445A606AE711F0030F1A
:1030500008BFD7F800808C4588BF02F8018B01F1CA
:10306000010188BF4FEA1828E3E700BFF82F0020CE
:10307000436D03EB4111D1F8003B43F40013C1F859
:10308000003B7047436D03EB4111D1F8003943F425
:103090000013C1F800397047436D03EB4111D1F8BB
:1030A000003B23F40013C1F8003B7047436D03EB72
:1030B0004111D1F8003923F40013C1F800397047E9
:1030C00000F1604303F561430901C9B283F80013BD
:1030D000012200F01F039A4043099B0003F1604363
:1030E00003F56143C3F880211A60704730B5039C33
:1030F0000172043304FB0325C0E90653049B0363F8
:103100000021059BC160C0E90000C0E90422C0E9BC
:103110000842C0E90A11436330BD0000416A002241
:10312000C0E90411C0E90A22C2606FF00101FEF794
:10313000E5BE0000D0E90432934201D1C2680AB969
:10314000181D70470020704703691960C26801327A
:10315000C260C269134482690361934224BF436A17
:1031600003610021FEF7BEBE38B504460D46E36894
:103170003BB16269131D1268A3621344E36200202D
:1031800007E0237A33B929462046FEF79BFE002844
:10319000EDDA38BD6FF00100FBE70000C368C269DB
:1031A000013BC3604369134482694361934224BF76
:1031B000436A436100238362036B03B1184770477E
:1031C00070B53023044683F31188866A3EB9FFF751
:1031D000CBFF054618B186F31188284670BDA36A57
:1031E000E26A13F8015BA362934202D32046FFF721
:1031F000D5FF002383F31188EFE700002DE9F84F96
:1032000004460E46174698464FF0300989F3118858
:103210000025AA46D4F828B0BBF1000F09D14146D9
:103220002046FFF7A1FF20B18BF311882846BDE8A7
:10323000F88FD4E90A12A7EB050B521A934528BF61
:103240009346BBF1400F1BD9334601F1400251F8C0
:10325000040B43F8040B9142F9D1A36A4033403682
:10326000A3624035D4E90A239A4202D32046FFF7ED
:1032700095FF8AF31188BD42D8D289F31188C9E736
:1032800030465A46FDF710FDA36A5B445E44A362D4
:103290005D44E7E710B5029C0172043303FB04218F
:1032A000C0E906130023C0E90A33039B0363049BB0
:1032B000C460C0E90000C0E90422C0E908424363D9
:1032C00010BD0000026AC260426AC0E90422002206
:1032D000C0E90A226FF00101FEF710BED0E9042315
:1032E0009A4201D1C26822B9184650F8043B0B60DB
:1032F000704700231846FAE7C368C2690133C36008
:103300004369134482694361934224BF436A436122
:103310000021FEF7E7BD000038B504460D46E3681E
:103320003BB123691A1DA262E2691344E3620020E3
:1033300007E0237A33B929462046FEF7C3FD00286B
:10334000EDDA38BD6FF00100FBE70000036919609A
:10335000C268013AC260C269134482690361934240
:1033600024BF436A036100238362036B03B11847E0
:103370007047000070B530230D460446114683F3B4
:103380001188866A2EB9FFF7C7FF10B186F311883E
:1033900070BDA36A1D70A36AE26A01339342A362FF
:1033A00004D3E16920460439FFF7D0FF002080F301
:1033B0001188EDE72DE9F84F04460D4690469946F1
:1033C0004FF0300A8AF311880026B346A76A4FB936
:1033D00049462046FFF7A0FF20B187F31188304609
:1033E000BDE8F88FD4E90A073A1AA8EB0607974216
:1033F00028BF1746402F1BD905F1400355F8042B71
:1034000040F8042B9D42F9D1A36A4033A3624036B1
:10341000D4E90A239A4204D3E16920460439FFF72C
:1034200095FF8BF311884645D9D28AF31188CDE7F1
:1034300029463A46FDF738FCA36A3B443D44A36263
:103440003E44E5E7D0E904239A4217D1C3689BB113
:10345000836A8BB1043B9B1A0ED01360C368013B97
:10346000C360C3691A44836902619A4224BF436AF4
:103470000361002383620123184670470023FBE7A2
:1034800000F036B9014B586A704700BF000C00408D
:10349000034B002258631A610222DA60704700BFB2
:1034A000000C0040014B0022DA607047000C004025
:1034B000014B5863704700BF000C0040FEE700005E
:1034C00070B51B4B01630025044686B058608562C9
:1034D0000E4600F0BFF804F11003C4E904334FF0C6
:1034E000FF33C4E90635C4E90044A560E562FFF78F
:1034F000C9FF2B460246C4E9082304F134010D4AF2
:10350000256580232046FEF793FC0123E0600A4AEC
:103510000375009272680192B268CDE90223074BED
:103520006846CDE90435FEF7ABFC06B070BD00BFC0
:1035300090280020983D00089D3D0008BD340008FB
:10354000024AD36A1843D062704700BF2826002081
:103550004B6843608B688360CB68C3600B694361D1
:103560004B6903628B6943620B680360704700001C
:1035700008B5264B26481A6940F2FF110A431A6122
:103580001A6922F4FF7222F001021A611A691A6B99
:103590000A431A631A6D0A431A651E4A1B6D1146C7
:1035A000FFF7D6FF02F11C0100F58060FFF7D0FFA6
:1035B00002F1380100F58060FFF7CAFF02F1540103
:1035C00000F58060FFF7C4FF02F1700100F5806034
:1035D000FFF7BEFF02F18C0100F58060FFF7B8FF36
:1035E00002F1A80100F58060FFF7B2FF02F1C4010B
:1035F00000F58060FFF7ACFF02F1E00100F58060AC
:10360000FFF7A6FFBDE8084000F0F0B80038024020
:1036100000000240A43D000808B500F069FAFEF77A
:10362000CBFBFFF78DF8BDE80840FEF753BE000066
:1036300070470000EFF3098305494A6B22F001024D
:103640004A63683383F30988002383F31188704742
:1036500000EF00E0302080F3118862B60C4B0D4A79
:10366000D96821F4E0610904090C0A43DA60D3F84F
:10367000FC20094942F08072C3F8FC200A6842F03D
:1036800001020A602022DA7783F82200704700BF27
:1036900000ED00E00003FA05001000E010B5302353
:1036A00083F311880E4B5B6813F4006314D0F1EEC2
:1036B000103AEFF30984683C4FF08073E361094BE3
:1036C000DB6B236684F30988FEF74AFB10B1064BD7
:1036D000A36110BD054BFBE783F31188F9E700BF39
:1036E00000ED00E000EF00E02F03000832030008C7
:1036F0000E4B1A6C42F008021A641A6E42F008026D
:103700001A660B4A1B6E936843F008039360094BDB
:1037100053229A624FF0FF32DA6200229A615A63B2
:10372000DA605A6001225A611A607047003802401C
:10373000002004E0000C0040094A08B51169D36874
:103740000B40D9B2C9439B07116107D5302383F3DE
:103750001188FEF747FB002383F3118808BD00BFE3
:10376000000C00401F4B1A696FEAC2526FEAD25236
:103770001A611A69C2F308021A614FF0FF301A6920
:103780005A69586100215A6959615A691A6A62F086
:1037900080521A621A6A02F080521A621A6A5A6ACF
:1037A00058625A6A59625A6A1A6C42F080521A6414
:1037B0001A6E42F080521A661A6E0B4A106840F474
:1037C00080701060186F00F44070B0F5007F1EBF6D
:1037D0004FF4803018671967536823F400735360FF
:1037E00000F05EB90038024000700040334B4FF0EB
:1037F00080521A64324A4FF4404111601A6842F014
:1038000001021A601A689107FCD59A6822F0030237
:103810009A602A4B9A6812F00C02FBD1196801F0E9
:10382000F90119609A601A6842F480321A601A68C5
:103830009203FCD55A6F42F001025A671F4B5A6F30
:103840009007FCD51F4A5A601A6842F080721A60CD
:103850001B4A53685904FCD5184B1A689201FCD5D1
:10386000194A9A60194B1A68194B9A42194B21D17F
:10387000194A1168194A91421CD140F205121A6086
:10388000144A136803F00F03052BFAD10B4B9A6807
:1038900042F002029A609A6802F00C02082AFAD1F9
:1038A0005A6C42F480425A645A6E42F480425A661C
:1038B0005B6E704740F20572E1E700BF00380240DE
:1038C000007000400854400700948838002004E04D
:1038D00011640020003C024000ED00E041C20F41B5
:1038E000074A08B5536903F00103536123B1054A40
:1038F00013680BB150689847BDE80840FFF7CEBE8B
:10390000003C014070300020074A08B5536903F0BD
:103910000203536123B1054A93680BB1D0689847FD
:10392000BDE80840FFF7BABE003C014070300020FF
:10393000074A08B5536903F00403536123B1054AEC
:1039400013690BB150699847BDE80840FFF7A6BE60
:10395000003C014070300020074A08B5536903F06D
:103960000803536123B1054A93690BB1D0699847A5
:10397000BDE80840FFF792BE003C014070300020D7
:10398000074A08B5536903F01003536123B1054A90
:10399000136A0BB1506A9847BDE80840FFF77EBE36
:1039A000003C014070300020164B10B55C6904F4F7
:1039B00078725A61A30604D5134A936A0BB1D06A90
:1039C0009847600604D5104A136B0BB1506B9847AB
:1039D000210604D50C4A936B0BB1D06B9847E205D6
:1039E00004D5094A136C0BB1506C9847A30504D554
:1039F000054A936C0BB1D06C9847BDE81040FFF7B7
:103A00004DBE00BF003C014070300020194B10B586
:103A10005C6904F47C425A61620504D5164A136D50
:103A20000BB1506D9847230504D5134A936D0BB124
:103A3000D06D9847E00404D50F4A136E0BB1506E59
:103A40009847A10404D50C4A936E0BB1D06E9847E9
:103A5000620404D5084A136F0BB1506F98472304D2
:103A600004D5054A936F0BB1D06F9847BDE810405D
:103A7000FFF714BE003C01407030002008B5034839
:103A8000FDF77CFABDE80840FFF708BEBC23002024
:103A900008B5FFF751FEBDE80840FFF7FFBD000085
:103AA000062108B50846FFF70BFB06210720FFF7A4
:103AB00007FB06210820FFF703FB06210920FFF77B
:103AC000FFFA06210A20FFF7FBFA06211720FFF76D
:103AD000F7FA06212820FFF7F3FA07213220FFF733
:103AE000EFFABDE808400C214720FFF7E9BA0000D3
:103AF00008B5FFF737FE00F00DF8FDF753FCFDF7B2
:103B000039FEFDF711FDFFF793FDBDE80840FFF713
:103B1000B7BC00000023054A19460133102BC2E947
:103B2000001102F10802F8D1704700BF7030002088
:103B3000034611F8012B03F8012B002AF9D1704735
:103B400053544D3332463F3F3F0053544D3332467A
:103B50003430780053544D33324634327800535465
:103B60004D333246343436585800000001203300BB
:103B70000010410001105A000310590007103100D5
:103B800000000000403B0008130400004A3B00080E
:103B900019040000543B0008210400005E3B0008AB
:103BA000009600000000000000000000000000007F
:103BB0000000000000000000651300085113000819
:103BC0008D1300087913000885130008711300088D
:103BD0005D13000849130008991300080000000055
:103BE000A514000891140008CD140008B9140008A9
:103BF000C5140008B11400089D14000889140008B9
:103C0000D9140008000000000100000000000000BE
:103C100063300000103C000880260020902800201F
:103C20004172647550696C6F740025424F41524473
:103C3000252D424C002553455249414C250000009A
:103C40000200000000000000C11600082D17000847
:103C500040004000302D0020402D002002000000D8
:103C600000000000030000000000000071170008C1
:103C70000000000010000000502D00200000000097
:103C80000100000000000000F82F002001010200E8
:103C900071220008812100081D220008012200086D
:103CA00043000000A83C000809024300020100C0D4
:103CB0003209040000010202010005240010010580
:103CC00024010001042402020524060001070582E4
:103CD000030800FF09040100020A000000070501B3
:103CE00002400000070581024000000012000000B1
:103CF000F43C000812011001020000400912415773
:103D000000020102030100000403090425424F419F
:103D10005244250051696F54656B41646570744667
:103D20003430370030313233343536373839414268
:103D300043444546000000000040000000400000F1
:103D400000400000004000000000010000000200F0
:103D5000000002000000020000000200000002005B
:103D6000000002000000020000000000B51800087A
:103D70006D1B0008191C000840004000583000204E
:103D80005830002001000000683000208000000052
:103D900040010000030000006D61696E0069646C01
:103DA000650000000000802A00000000AAAAAAAA5C
:103DB00000000024FFFF00000000000000A00A0037
:103DC0004000000000000000AAAAAAAA40000000CB
:103DD000FFFF0000000000000000000000A0000441
:103DE00000000000AAAAAAA200500004FFFF0000E1
:103DF00000000088000000004041000000000000BA
:103E0000AAAAAAAA40410000FFFF0000000000008B
:103E1000000000000011004100000000AAAAAAAAA8
:103E200000110000FFFF0000000000000000000083
:103E30000000000000000000AAAAAAAA00000000DA
:103E4000FFFF000000000000000000000000000074
:103E500000000000AAAAAAAA00000000FFFF0000BC
:103E60000000000000000000000000000000000052
:103E70000A00000000000000030000000000000035
:103E80000000000000000000000000000000000032
:103E90000000000000000000000000000000000022
:103EA000290400000000000000C00F000000000016
:103EB000FF00000098280020BC230020009600008E
:103EC0000000080096000000000800000400000048
:103ED000083D000800000000000000000000000095
:0C3EE000000000000000000000000000D6
:00000001FF
